:020000040000FA
:1000000083160313023086001930990000309800DF
:100010009F008312031307309F0000309A0099005D
:10002000A000A100903098008C1E14281A08A1008E
:100030000311533C0319252821084C3C031935288A
:100040002108523C03197C28912821085320203094
:10005000532083160313FF30850083120313982067
:100060000D3053200A30532014282108532020300B
:1000700053200430A200A8018C1E3C281A08A000BE
:100080000311303C031949282008313C0319492841
:100090003C285D20A20B3C2868206F200D305320A7
:1000A0000A30532014289900831603139816981CBD
:1000B000572800008312031308001A08A0005320D9
:1000C000201C65280314A80D08000310A80D0800C3
:1000D0000430A2000310A80DA20B6A28080006082D
:1000E0000F3928048600752008000430A700583016
:1000F0005320A70B772808000000831603133E3017
:1001000085008312031321085320A31C8A28A310FF
:1001100005108C28A31405140D3053200A305320E9
:100120001428463053200D3053200A305320142811
:100130000830A2008030A700A00003112008A7000B
:100140000508A705031DA528AC283130532003104E
:10015000A00CA20B9D281428303053200310A00CB3
:10016000A20B9D2808001030A400FF30A500FF302E
:10017000A600A60BB928A50BB728A40BB528080024
:02400E00293F48
:00000001FF
